:100000000C94480D0C94790D0C94790D0C94790D89
:100010000C94790D0C94790D0C94790D0C94790D48
:100020000C94790D0C94790D0C94790D0C94790D38
:100030000C94790D0C94790D0C94790D0C94790D28
:100040000C94790D0C948D850C94790D0C94790D8C
:100050000C94790D0C94790D0C94790D0C94DFB7F8
:100060000C94790D0C9458BB0C948EBB0C94790DA8
:100070000C94790D0C94790D0C94790D0C94790DE8
:100080000C94BA850C94790D0C94790D0C94790D1F
:100090000C94790D0C94790D0C94790D0C94790DC8
:1000A0000C94790D0C94790D0C94E7850C94790DD2
:1000B0000C94790D0C94790D0C94790D0C94148694
:1000C0000C94790D0C94790D0C94790D0C94790D98
:1000D0000C94790D0C94790D0C94790D0C94790D88
:1000E0000C94790DDC16DB172A1878189318AE18C3
:1000F000C918FC18721A451A5C192F19371E371EB9
:100100008D19A819371EBA1A8D1AB11BAE1C811C85
:100110000E1DE11C681B4D1B1A1BED1A1B1CCC1B72
:100120004E1C0F174217C319121A45187517371EA0
:10013000121ACE1DA11D6E1D411DA817011EA16121
:10014000A965A461A861A965AD61B361B961E56103
:10015000A163C963A965A965F1635563A9651362C4
:100160003F62026404642D64596482646D62936228
:10017000DB620363FA63F863FC6399619D619263D8
:10018000FE63AE644763A9650064C664F8642965CC
:100190005A65B2648A652E7E357E3C7E437E4A7EF9
:1001A000617E517E617E587ED17ED57ED97EDD7E98
:1001B000E17EE57EE97E178F358F5C8F728F728FBF
:1001C000728F898F1190178F1190AC8F1190BA8F09
:1001D000BA8FD78FD78F5C8F3D903D905C8FBA8F51
:1001E0001190728FE58F11901190119011901190D4
:1001F000FF8F11901190AA900B92F492C393CE941A
:10020000CE946096B497599DC198B29A1E9BE79E72
:10021000C09F9CA19CA1F4928FAA8FAAF49293A054
:100220009DA2E29566A331A437A65EA5F0A637A8E5
:1002300091A9A5A9599916B919B908B90CB912B952
:1002400050B91DB921B927B92BB92FB935B939B969
:100250003DB950B943B947B94BB905A84CCDB2D453
:100260004EB93836A9020C50B9918688083CA6AA26
:10027000AA2ABE000000803F50424D20696D616790
:1002800065206D757374206265206174206C6561F2
:10029000737420313020706978656C7320776964DD
:1002A000652E002C206D61782064656E7369747909
:1002B0003A20002C2070656E2077696474683A20BB
:1002C0000050656E776964746820746573742000EB
:1002D0002C20726564756365643A002C206F757418
:1002E0004D61783A002C20696E4D61783A00696E54
:1002F00044656E733A004E6F7420706F7373696259
:100300006C6520746F206578707265737320616E00
:10031000792064657461696C2E0020697320002C5B
:1003200020677269643A20004D61782077617665B4
:100330007320666F722070656E53697A653A20008B
:100340002C20736F20726F7773697A6520696E2035
:1003500073746570733A20002C206D6D5065725374
:100360007465703A2000472C442C726F7773697A59
:100370006520696E206D6D3A20002073746570737E
:100380002E003A20004D696E207365676D656E74AE
:100390002073697A6520666F722070656E53697A82
:1003A00065200063616C632053450063616C6320CA
:1003B0004E570063616C632053570063616C632088
:1003C0004E450063616C63756C61746564204E45D5
:1003D0000063616C63756C617465642053570063DE
:1003E000616C63756C617465642053450063616C76
:1003F00063756C61746564204E57002E002C207369
:100400006F75726365423A20002E20536F757263D8
:1004100065413A20002C20746172676574423A206D
:1004200000546172676574413A20002C206F4F754B
:1004300074206E756D626572206F662077617665D7
:10044000733A20002C20696E7075742064656E7399
:100450006974793A20004D61782077617665732060
:100460007769746820746869732070656E20616EA6
:1004700064206772696473697A653A20002E002EE1
:1004800020656E6420706F696E743A200053746149
:10049000727420706F696E743A2000643A204E4581
:1004A00000643A204E5700643A20535700643A20C3
:1004B0005345002C206D61782064656E73697479F2
:1004C0003A20002C2070656E2077696474683A20A9
:1004D0000050656E776964746820746573742000D9
:1004E0004368616E67696E67206261636B20746F39
:1004F000206C697665206D6F64652E0046696C65B9
:100500002072656D6F7665642E0046696C652061AA
:100510006C7265616479206578697374732E004527
:100520007865637574696E6720636F6D6D616E6465
:100530003A0053746F72696E6720636F6D6D616E00
:10054000643A006D6D004368616E676564205065B4
:100550006E20776964746820746F20004E65772080
:10056000616363656C65726174696F6E3A20004EF9
:100570006577206D61782073706565643A20005559
:10058000703A2000446F776E3A2000504753504530
:1005900045442C0050474C4946542C005047535476
:1005A00045504D554C5449504C4945522C005047EC
:1005B00053544550535045525245562C0050474DC8
:1005C0004D5045525245562C00504753495A452CE0
:1005D0000050474E414D452C002900526563616C27
:1005E00063207061676548656967687420696E207B
:1005F00073746570732028002900526563616C6311
:100600002070616765576964746820696E2073742F
:100610006570732028002900292C2073746570737D
:100620005065724D4D202800526563616C63206DEA
:100630006D506572537465702028004C6F6164655D
:1006400064206D6F746F722073746570206D756CAB
:100650007469706C6965723A004C6F6164656420FE
:100660006D616368696E65206E616D653A004C6FFF
:100670006164656420757020706F733A004C6F611F
:1006800064656420646F776E20706F733A004C6FFE
:1006900061646564206D6F746F722073746570732C
:1006A00020706572207265763A004C6F61646564F3
:1006B000206D6D20706572207265763A004C6F6116
:1006C000646564206D616368696E6520686569674B
:1006D00068743A004C6F61646564206D6163686999
:1006E0006E652077696474683A00206E6F742072BA
:1006F00065636F676E697365642E00506172616D2A
:10070000733A002C2070343A002C2070333A002CBD
:100710002070323A002C2070313A00436F6D6D61C9
:100720006E643A003A002D00503A2000496E3A209B
:1007300000325375623A200034696E533A20003219
:10074000696E533A200031696E533A200029206EB9
:100750006F74207061727365642E00436F6D6D203D
:100760002800786275663A2000427566706F733AA9
:1007700020006275663A20005465726D276400633C
:10078000683A200054696D6564206F75743A002ED4
:10079000002E2E2E004C61737420636F6D6D3A2015
:1007A00000536572766F20004861726477617265EC
:1007B0003A20007600504F4C415247524150482059
:1007C0004F4E21007C3C3E5E2B3D3F2F5B5D3B2C22
:1007D0002A225C001010205F0000000000000000D2
:1007E0000000000000000000000000000000000009
:1007F00000000000000000000000000007000F8063
:100800000F800F800F800F8007000700000000009E
:10081000070007000700000000000E380E380E38F1
:100820000E3806300000000000000000000000004C
:10083000000000000000000000000C300C300C3004
:100840007FFE7FFE0C300C300C300C307FFE7FFEC4
:100850000C300C300C3000000000024002400FF859
:100860001FF81A401A401FF00FF8025802581FF8DC
:100870001FF00240024000000000000000000E10C7
:100880000E300E7000E001C0038007000E700C7087
:100890000870000000000000000000000F00198038
:1008A000198019800F000F080F9819F818F018E038
:1008B00019F00F980000000000000000070007007A
:1008C00007000E0000000000000000000000000013
:1008D00000000000000000000000000000F001C067
:1008E000038007000E000E000E000E0007000380BC
:1008F00001C000F000000000000000000F000380B5
:1009000001C000E0007000700070007000E001C0E5
:1009100003800F000000000000000000018011882B
:10092000099007E007E03FFC3FFC07E007E0099083
:10093000118801800000000000000000000000009D
:100940000180018001800FF00FF0018001800180A3
:100950000000000000000000000000000000000097
:100960000000000000000000000000000000070080
:10097000070007000E00000000000000000000005B
:100980000000000000001FF81FF800000000000039
:100990000000000000000000000000000000000057
:1009A0000000000000000000000000000000070040
:1009B0000700070000000000000000000002000621
:1009C000000E001C0038007000E001C0038007002A
:1009D0000E001C0000000000000000000FF01C389A
:1009E0001C781CF81CF81DB81DB81F381F381E389D
:1009F0001C380FF0000000000000000001800180A2
:100A000003801F801F800380038003800380038096
:100A100003801FF000000000000000000FE01C70C9
:100A20001C380038007000E001C0038007000E3859
:100A30001C381FF800000000000000000FE01C70D0
:100A40001C380038007003C003C0007000381C3828
:100A50001C700FE0000000000000000000E001E05A
:100A600003E006E00CE018E01FF81FF800E000E0EB
:100A700000E003F800000000000000001FF81C0068
:100A80001C001C001C001FE01FF0007800381C3800
:100A90001C700FE0000000000000000003E00700F1
:100AA0000E001C001C001FF01FF81C381C381C38DE
:100AB0001C380FF000000000000000001FFC1C1C90
:100AC0001C1C1C1C001C0038007000E001C00380CE
:100AD0000380038000000000000000000FF01C38BD
:100AE0001C381C381F3807E007E01CF81C381C387D
:100AF0001C380FF000000000000000000FF01C3850
:100B00001C381C381C381FF80FF8003800380070EB
:100B100000E007C00000000000000000000000002E
:100B200003800380038000000000038003800380B3
:100B300000000000000000000000000000000000B5
:100B40000380038003800000000003800380038093
:100B500007000000000000000000007000E001C07D
:100B6000038007000E001C001C000E00070003801D
:100B700001C000E000700000000000000000000064
:100B800000003FFC3FFC000000003FFC3FFC000079
:100B9000000000000000000000001C000E00070024
:100BA000038001C000E00070007000E001C003801D
:100BB00007000E001C000000000003C00FF01E78AC
:100BC00018380038007000E001C001C000000000CB
:100BD00001C001C001C0000000000FF81C1C1C1C5B
:100BE0001C1C1C1C1CFC1CFC1CFC1CFC1C001C00FD
:100BF0001C001FF007F800000000000003C007E021
:100C00000E701C381C381C381C381FF81C381C3857
:100C10001C381C3800000000000000001FF00E38D7
:100C20000E380E380E380FF00FF00E380E380E3822
:100C30000E381FF0000000000000000007F00E3822
:100C40001C381C001C001C001C001C001C001C3854
:100C50000E3807F000000000000000001FE00E70DA
:100C60000E380E380E380E380E380E380E380E3854
:100C70000E701FE000000000000000001FF80E18BA
:100C80000E080E000E300FF00FF00E300E000E08A2
:100C90000E181FF800000000000000001FF80E18DA
:100CA0000E080E000E300FF00FF00E300E000E008A
:100CB0000E001F00000000000000000007F00E38CA
:100CC0001C381C381C001C001C001CF81C381C386C
:100CD0000E3807F800000000000000001C701C70B7
:100CE0001C701C701C701FF01FF01C701C701C709E
:100CF0001C701C7000000000000000000FE003806A
:100D000003800380038003800380038003800380CB
:100D100003800FE0000000000000000001FC0070F4
:100D2000007000700070007000703870387038709B
:100D300038700FE000000000000000001E380E3880
:100D40000E700EE00FC00F800F800FC00EE00E700F
:100D50000E381E3800000000000000001F000E00CA
:100D60000E000E000E000E000E000E000E080E18F3
:100D70000E381FF800000000000000001C1C1E3C84
:100D80001F7C1FFC1FFC1DDC1C9C1C1C1C1C1C1C39
:100D90001C1C1C1C00000000000000001C1C1C1C73
:100DA0001E1C1F1C1F9C1DDC1CFC1C7C1C3C1C1CDA
:100DB0001C1C1C1C000000000000000003E007F0E9
:100DC0000E381C1C1C1C1C1C1C1C1C1C1C1C0E3847
:100DD00007F003E000000000000000001FF00E38E4
:100DE0000E380E380E380FF00FF00E000E000E0009
:100DF0000E001F00000000000000000003E00F785C
:100E00000E381C1C1C1C1C1C1C1C1C7C1CFC0FF805
:100E10000FF8003800FC0000000000001FF00E3842
:100E20000E380E380E380FF00FF00E700E380E38E8
:100E30000E381E3800000000000000000FF01C38C3
:100E40001C381C381C000FE007F000381C381C3818
:100E50001C380FF000000000000000001FFC19CC3F
:100E600011C401C001C001C001C001C001C001C066
:100E700001C007F000000000000000001C701C70A2
:100E80001C701C701C701C701C701C701C701C7002
:100E90001C700FE000000000000000001C701C70BF
:100EA0001C701C701C701C701C701C701C700EE080
:100EB00007C0038000000000000000001C1C1C1C78
:100EC0001C1C1C1C1C1C1C9C1C9C1C9C0FF80FF844
:100ED0000770077000000000000000001C701C700C
:100EE0001C700EE007C00380038007C00EE01C707A
:100EF0001C701C7000000000000000001C701C70C2
:100F00001C701C701C700EE007C0038003800380FF
:100F100003800FE000000000000000001FF81C38F4
:100F20001838107000E001C0038007000E081C187C
:100F30001C381FF8000000000000000007F0070048
:100F40000700070007000700070007000700070069
:100F5000070007F00000000000000000100018006B
:100F60001C000E000700038001C000E00070003884
:100F7000001C0007000000000000000007F00070E7
:100F800000700070007000700070007000700070E1
:100F9000007007F0000000000000018003C007E0BF
:100FA0000E701C380000000000000000000000006F
:100FB0000000000000000000000000000000000031
:100FC0000000000000000000000000000000000021
:100FD000000000007FFF7FFF000000001C001C00DD
:100FE00007000700000000000000000000000000F3
:100FF00000000000000000000000000000000000F1
:10100000000000000FE0007000700FF01C701C70FA
:101010001C700FD800000000000000001E000E0031
:101020000E000E000FF00E380E380E380E380E3847
:101030000E381BF00000000000000000000000005F
:10104000000000000FE01C701C701C001C001C70D5
:101050001C700FE0000000000000000000F80070AD
:10106000007000700FF01C701C701C701C701C70E5
:101070001C700FD8000000000000000000000000FD
:10108000000000000FE01C701C701FF01C001C70A2
:101090001C700FE0000000000000000003E007707B
:1010A0000770070007001FE01FE0070007000700A8
:1010B00007001FC00000000000000000000000004A
:1010C000000000000FD81C701C701C701C700FF00A
:1010D00007F000701C700FE0000000001E000E0002
:1010E0000E000E000EF00F380F380E380E380E3886
:1010F0000E381E38000000000000000001C001C0D2
:1011000001C000000FC001C001C001C001C001C08A
:1011100001C00FF800000000000000000070007027
:101120000070000003F0007000700070007000702C
:1011300000701C700CF007E0000000001E000E00A4
:101140000E000E000E380E700EE00FC00EE00E7096
:101150000E381E3800000000000000000FC001C063
:1011600001C001C001C001C001C001C001C001C077
:1011700001C00FF8000000000000000000000000A7
:10118000000000001FF81C9C1C9C1C9C1C9C1C9CB0
:101190001C9C1C9C000000000000000000000000DF
:1011A000000000001FE01C701C701C701C701C7084
:1011B0001C701C7000000000000000000000000017
:1011C000000000000FE01C701C701C701C701C7074
:1011D0001C700FE000000000000000000000000094
:1011E000000000001BF00E380E380E380E380E3896
:1011F0000FF00E000E001F000000000000000000B5
:10120000000000001FB038E038E038E038E038E097
:101210001FE000E000E001F000000000000000001E
:10122000000000001EF00FF80F380E000E000E0038
:101230000E001F0000000000000000000000000081
:10124000000000000FE01C301C300F8003E018701D
:1012500018700FE000000000000000000000010016
:10126000030007001FF007000700070007000770D2
:10127000077003E000000000000000000000000014
:10128000000000001C701C701C701C701C701C7016
:101290001C700FD8000000000000000000000000DB
:1012A000000000001C701C701C701C701C700EE094
:1012B00007C00380000000000000000000000000E4
:1012C000000000001C1C1C1C1C1C1C9C1C9C0FF8FF
:1012D0000770077000000000000000000000000020
:1012E000000000001CE01CE00FC0078007800FC05A
:1012F0001CE01CE0000000000000000000000000F6
:10130000000000000E380E380E380E380E3807F088
:1013100003E000E001C01F800000000000000000AA
:10132000000000001FE018E011C0038007000E203D
:101330001C601FE0000000000000000001F80380B6
:101340000380038007001C001C000700038003804B
:10135000038001F800000000000001C001C001C0CE
:1013600001C001C001C001C001C001C001C001C075
:1013700001C001C001C00000000000001F8001C0CA
:1013800001C001C000E00038003800E001C001C029
:1013900001C01F8000000000000000001F1C3B9CDB
:1013A00039DC38F8000000000000000000000000F8
:1013B0000000000000000000080C205F000000009A
:1013C000000000000000000000002020202020205D
:1013D0000020000000285050000000000000000025
:1013E00000002828FC2850FC50500000002078A85D
:1013F000A0603028A8F02000000048A8B050283491
:1014000054480000000020505078A8A8906C0000BC
:1014100000404080000000000000000000040810B0
:1014200010101010100804000040201010101010B0
:101430001020400000000020A87070A820000000CC
:101440000000202020F820202000000000000000E4
:1014500000000000004040800000000000F8000094
:10146000000000000000000000000000004000003C
:1014700000081010102020404040800000007088BC
:101480008888888888700000000020602020202044
:1014900020700000000070888810204080F8000054
:1014A00000007088083008088870000000001030C4
:1014B00050509078101800000000F88080F0080864
:1014C000887000000000709080F0888888700000AC
:1014D0000000F890102020202020000000007088DC
:1014E0008870888888700000000070888888780874
:1014F00048700000000000002000000000200000F4
:10150000000000000020000000202000000408105F
:10151000204020100804000000000000F80000F83F
:1015200000000000004020100804081020400000C7
:1015300000007088881020200020000000007088C3
:1015400098A8A8B88078000000002020305050787B
:1015500048CC00000000F0484870484848F00000BF
:101560000000788880808080887000000000F0484B
:101570004848484848F000000000F8485070504083
:1015800048F800000000F8485070504040E000006B
:101590000000384880809C88483000000000CC481B
:1015A0004878484848CC00000000F820202020203F
:1015B00020F8000000007C10101010101090E000C7
:1015C0000000EC485060505048EC00000000E04043
:1015D0004040404044FC00000000D8D8D8D8A8A81B
:1015E000A8A800000000DC486868585848E80000D7
:1015F0000000708888888888887000000000F048A3
:101600004870404040E0000000007088888888E80A
:10161000987018000000F0484870504848EC0000EE
:10162000000078888060100888F000000000F8A8AA
:1016300020202020207000000000CC484848484866
:10164000483000000000CC484850503020200000B6
:101650000000A8A8A8705050505000000000D850BA
:101660005020205050D800000000D850502020209A
:10167000207000000000F8901020204048F8000082
:10168000003820202020202020203800004040402A
:101690002020101010080000007010101010101002
:1016A000101070000020500000000000000000003A
:1016B0000000000000000000000000FC002000000E
:1016C000000000000000000000000000003048386A
:1016D000483C00000000C04040704848487000008E
:1016E00000000000003848404038000000001808A2
:1016F00008384848483C00000000000000304878A6
:101700004038000000001C202078202020780000B5
:1017100000000000003C4830407844380000C040E1
:101720004070484848EC0000000020000060202085
:10173000207000000000100000301010101010E0A9
:101740000000C040405C507048EC00000000E02009
:101750002020202020F800000000000000F0A8A8B1
:10176000A8A800000000000000F0484848EC000075
:101770000000000000304848483000000000000031
:1017800000F04848487040E0000000000038484839
:101790004838081C0000000000D8604040E000000D
:1017A00000000000007840300878000000000020B1
:1017B00020702020201800000000000000D84848B9
:1017C000483C00000000000000EC485030200000C1
:1017D0000000000000A8A8705050000000000000A9
:1017E00000D8502050D800000000000000EC485005
:1017F000302020C000000000007810202078000079
:1018000000181010102010101010180010101010D8
:101810001010101010101010006020202010202038
:101820002020600040A4180000000000000000001C
:1018300000000A0B02090C0D0E080703040100004A
:101840000000000000000000000000000000000098
:101850000000000000000000000000001211100055
:101860000000000000000000000000000000000078
:101870000000000000000102102020080810204095
:101880001020408002010201080402010102040844
:1018900010204080804020100804020180040201D2
:1018A000804020100804020108040201010204081B
:1018B0001020408001020408102040800505050525
:1018C000070508080808020202020A0A08080404B8
:1018D00004040101010101010101030303030303E6
:1018E0000303040707070C0C0C0C0C0C0C0C020275
:1018F000020206060606060606060B0B0B0B0B0B72
:101900000B0B000020002300260029002C002F00D4
:10191000320000010000030106010901000022005D
:10192000250028002B002E003100340002010000A9
:10193000050108010B0100002100240027002A00F6
:101940002D003000330001010000040107010A01ED
:101950004E414E494E495459494E46CDCCCC3D0A94
:10196000D7233C17B7D13877CC2B329595E6241F77
:10197000B14F0A000020410000C84200401C462030
:10198000BCBE4CCA1B0E5AAEC59D7400407A10F303
:101990005A00A0724E18090010A5D4E80000E8769D
:1019A00048170000E40B54020000CA9A3B000000F4
:1019B000E1F505000080969800000040420F00000D
:1019C00000A08601000000102700000000E80300CE
:1019D0000000006400000000000A00000000000198
:1019E00000000000002C76D888DC674F0823DFC198
:1019F000DFAE59E1B1B796E5E3E453C63AE6519953
:101A00007696E8E6C28426EB898C9B62ED407C6F7B
:101A1000FCEFBC9C9F40F2BAA56FA5F490055A2A32
:101A2000F75C936B6CF9676DC11BFCE0E40D47FE3E
:101A3000F520E6B500D0ED902E0300943577050033
:101A400080841E080000204E0A000000C80C3333BA
:101A500033330F986E12831141EF8D2114893BE6C9
:101A60005516CFFEE6DB18D1844B381BF77C1D9052
:101A70001DA4BBE424203284725E228100C9F124BB
:101A8000ECA1E53D27007038D36EE471C0BB5C3A31
:101A900011241FBECFEFD1E2DEBFCDBF00E00CBFEF
:101AA00012E1A0E0B2E0E4E0FAE901E00BBF02C01D
:101AB00007900D92A239B107D9F729E1A2E9B2E165
:101AC00001C01D92A13AB207E1F71AE1CEE8DAE1CE
:101AD00000E006C022970109FE010BBF0E947EC5EF
:101AE000C638D10780E00807A9F70E94D1C10C943D
:101AF000F1CC0C9400000E94EAC091E0811190E0CA
:101B0000892F0895CF92DF92EF92FF920F931F9348
:101B1000CF93DF93CDB7DEB7EDB6FEB6FC010190F3
:101B20000020E9F73197E81BF90B2DB73EB72E1BC4
:101B30003F0B0FB6F8943EBF0FBE2DBF0DB71EB7BB
:101B40000F5F1F4FBC01C8010E947EC88091F6152F
:101B5000882389F06CE277E08DEF98E10E9441BC28
:101B6000B8018DEF98E10E9472BC63E373E08DEFE2
:101B700098E10E949DBC6EE372E1C8010E9451C8C9
:101B80008C011092B3151092A51510929715109212
:101B90008915D12CC12CD11004C0B80181EC95E17C
:101BA0003CC06EE372E180E090E00E9451C88C017D
:101BB000009741F0BC0189E392E10E94A2C8892B01
:101BC00009F4C39432E0D316A1F03D1520F081E072
:101BD000D81641F024C023E0D21691F034E0D31699
:101BE000B1F01DC001151105D1F0B80183EB95E1ED
:101BF00014C00115110599F0B80185EA95E10DC0F1
:101C00000115110561F0B80187E995E106C00115DC
:101C1000110529F0B80189E895E10E947EC88091FC
:101C2000F615882329F168E277E08DEF98E10E94AC
:101C300041BC4AE050E06D2D8DEF98E10E948BBDD4
:101C400066E277E08DEF98E10E9441BC4AE050E007
:101C50006C2D8DEF98E10E948BBD64E277E08DEFF3
:101C600098E10E9441BCB8018DEF98E10E949DBCB3
:101C7000D39486E0D8128FCFC09288158091F61544
:101C8000882309F44AC06BE177E08DEF98E10E9468
:101C900041BC61EC75E18DEF98E10E9472BC65E199
:101CA00077E08DEF98E10E9441BC63EB75E18DEF29
:101CB00098E10E9472BC6FE077E08DEF98E10E949E
:101CC00041BC65EA75E18DEF98E10E9472BC69E064
:101CD00077E08DEF98E10E9441BC67E975E18DEFF7
:101CE00098E10E9472BC63E077E08DEF98E10E947A
:101CF00041BC69E875E18DEF98E10E949DBC6BEFF6
:101D000076E08DEF98E10E9441BC4AE050E060919E
:101D100088158DEF98E10E9491BD0FB6F894FEBE34
:101D20000FBEEDBEDF91CF911F910F91FF90EF900D
:101D3000DF90CF9008950F931F93CF93DF93EC0123
:101D40008091F615882359F066E477E08DEF98E1ED
:101D50000E9441BCBE018DEF98E10E949DBC69E3E9
:101D600072E1CE010E94A2C88C018091F6158823F1
:101D700059F06FE377E08DEF98E10E9441BCBE011E
:101D80008DEF98E10E949DBCF80114828091F615B8
:101D9000882311F168E377E08DEF98E10E9441BC60
:101DA000BE018DEF98E10E949DBC61E377E08DEF6D
:101DB00098E10E9441BCB8018DEF98E10E949DBC62
:101DC00069E372E1C8010E9475C84AE050E0BC01B5
:101DD0008DEF98E10E9459BD69E372E1C8010E944C
:101DE00075C8892B21F4CE018DDE81E001C080E031
:101DF000DF91CF911F910F91089566E475E18DEF0A
:101E000098E10C948DBCCF93DF93EC0165E572E013
:101E10008DEF98E10E9472BCBE018DEF98E10E94A7
:101E200064BC6AEE76E08DEF98E1DF91CF910C947F
:101E30007DBC61E083E00E9451B961E083E00E94D3
:101E40008AB961E086E00E9451B961E086E00E94B3
:101E50008AB963E08BE093E10E947E8421E040E058
:101E600060E08BE093E10E94938466E087EC92E16E
:101E70000E947E8421E040E061E087EC92E10C94D6
:101E80009384CF93DF93C0E0D0E04AE050E0BE01FE
:101E90008DEF98E10E9452BD67E373E08DEF98E10A
:101EA0000E9472BCCE010E9400C94AE050E0682F37
:101EB0008DEF98E10E9491BD2196C832D10529F796
:101EC000DF91CF910895FF920F931F93CF93DF93EC
:101ED000CDB7DEB72C970FB6F894DEBF0FBECDBFDF
:101EE00069E278E0CE0107960E94AEBF04E010E000
:101EF000C8010E9400C9F82EBE01695F7F4FCE0164
:101F000001960E940DC06F2DCE0101960E949DC0CA
:101F1000BC01CE0107960E94F8BFCE0101960E9437
:101F200046BF0F5F1F4F0C30110511F760E070E0E6
:101F3000CE0107960E9439C1FC018081811106C043
:101F40006FED75E1CE0107960E94F8BF1092CB1598
:101F50001092CC151092CD151092CE15BE01695F6E
:101F60007F4F85EE95E10E94F8BF69E576E08DEF41
:101F700098E10E9441BC65EE75E18DEF98E10E9409
:101F80008DBCCE0107960E9446BF2C960FB6F894E2
:101F9000DEBF0FBECDBFDF91CF911F910F91FF909C
:101FA000089583EB95E10E9406C890935D028093AB
:101FB0005C0285EA95E10E9406C890935F028093D7
:101FC0005E0208955EDF61ED75E08DEF98E10E949D
:101FD00041BC65EE75E18DEF98E10E9464BC69E358
:101FE00072E18DEF98E10E949DBC69EC75E08DEF88
:101FF00098E10E9441BC6091790270917A024AE0B6
:1020000050E08DEF98E10E9452BD6EE372E18DEFDA
:1020100098E10E9472BC60917702709178024AE068
:1020200050E08DEF98E10E9452BD69E372E18DEFBF
:1020300098E10E949DBC6DEB75E08DEF98E10E94E8
:1020400041BC409185025091860260918702709157
:10205000880222E030E08DEF98E10E948DBE69E3B6
:1020600072E18DEF98E10E949DBC6EEA75E08DEF04
:1020700098E10E9441BC6091890270918A024AE015
:1020800050E08DEF98E10E9452BD69E372E18DEF5F
:1020900098E10E949DBC6CE975E08DEF98E10E948B
:1020A00041BC60918302709184024AE050E08DEF60
:1020B00098E10E9452BD69E372E18DEF98E10E94C0
:1020C0009DBC64E975E08DEF98E10E9441BC609190
:1020D0008B0270918C024AE050E08DEF98E10E94F3
:1020E00052BD6EE372E18DEF98E10E9472BC609187
:1020F0008D0270918E024AE050E08DEF98E10E94CF
:1021000052BD69E372E18DEF98E10E949DBC6BE8DE
:1021100075E08DEF98E10E9441BC409173025091AF
:102120007402609175027091760222E030E08DEFCA
:1021300098E10E948DBE6EE372E18DEF98E10E94FE
:1021400072BC40916F025091700260917102709167
:10215000720222E030E08DEF98E10E948DBE69E3CB
:1021600072E18DEF98E10C949DBCAB01BC014093F2
:1021700073025093740260937502709376028BE041
:1021800093E10E94728340917302509174026091B6
:1021900075027091760287EC92E10E9472836FE67D
:1021A00075E08DEF98E10E9441BC4091730250911F
:1021B0007402609175027091760222E030E08DEF3A
:1021C00098E10C948EBEAB01BC0140936F0250931A
:1021D000700260937102709372028BE093E10E942F
:1021E000D68340916F02509170026091710270919C
:1021F000720287EC92E10E94D6836CE575E08DEF68
:1022000098E10E9441BC40916F0250917002609130
:1022100071027091720222E030E08DEF98E10C942F
:102220008EBE4F925F926F927F928F929F92AF92EB
:10223000BF92CF92DF92EF92FF920F931F93CF93B3
:10224000DF93CDB7DEB728970FB6F894DEBF0FBE89
:10225000CDBF6D837E838F83988749015A016701C3
:102260007801672B682B692B09F498C0C501B4016C
:102270000E94D3C32B013C0120E030E0A901C5013D
:10228000B4010E9444C287FF04C077FA709477F8C3
:102290007094A7019601C701B6010E94E0C169834D
:1022A0007A838B839C839B01AC01C301B2010E94A2
:1022B0004BC22B013C016D817E818F8198850E94EC
:1022C000E6C29B01AC01C301B2010E9444C240902E
:1022D000730250907402609075027090760220E054
:1022E00030E0A90187FF25C0C501B4010E9444C2A6
:1022F000811107C069817A818B819C810E9440C4D1
:102300000DC0A5019401C701B6010E944BC29B01FB
:10231000AC015F77C501B4010E94E0C16B017C0193
:10232000A30192010E94CFC318169CF12601370128
:1023300030C0C501B4010E9444C281110DC0698141
:102340007A818B819C810E9440C46B017C01F7FAE9
:10235000F094F7F8F0940FC0A5019401C701B601FD
:102360000E944BC29B01AC015F77C501B4010E9482
:10237000DFC16B017C0177FA709477F87094A30148
:102380009201C701B6010E9444C287FD02C0260126
:102390003701542D452D362D272D04C050E040E047
:1023A00030E020E0652F742F832F922F28960FB6F0
:1023B000F894DEBF0FBECDBFDF91CF911F910F917B
:1023C000FF90EF90DF90CF90BF90AF909F908F9055
:1023D0007F906F905F904F900895CF92DF92EF9231
:1023E000FF920F931F93CF93DF93CDB7DEB72C9758
:1023F0000FB6F894DEBF0FBECDBFEDB6FEB663EBF1
:1024000075E1CE0107960E94AEBF65EA75E1CE0187
:1024100001960E94AEBF69E278E0CE0107966BDBC1
:10242000882309F45AC06AE373E08DEF98E10E94B3
:1024300072BCBE01695F7F4F8DEF98E10E948DBC39
:1024400081E08093AF13BE01695F7F4F89EA93E11A
:102450000E94F8BF6FEC74E0CE0101960E94EAC0C2
:10246000882309F440C0CDB6DEB64B855C854F5F4E
:102470005F4F8DB79EB7841B950B0FB6F8949EBF28
:102480000FBE8DBF0DB71EB70F5F1F4F20E030E0AE
:10249000B801CE0107960E944BC1B8018AE096E1CF
:1024A0000E94476E882399F06AE075E08DEF98E10D
:1024B0000E947DBCB8018AE096E10E94516E88239B
:1024C00031F06CEF74E08DEF98E10E947DBC0FB6A7
:1024D000F894DEBE0FBECDBE06C067E573E08DEF9B
:1024E00098E10E949DBCCE0101960E9446BFCE019C
:1024F00007960E9446BF0FB6F894FEBE0FBEEDBE13
:102500002C960FB6F894DEBF0FBECDBFDF91CF91F2
:102510001F910F91FF90EF90DF90CF90089560EEA4
:1025200074E08DEF98E10E947DBC1092AF13089586
:1025300083EB95E10E9406C8009719F0019721F0FE
:1025400008951092F615089581E08093F615089588
:102550000F931F93CF93DF938091BD13811153C0CD
:102560008EEB93E10E946AB6882309F456C08EEB85
:1025700093E10E94CAB48EEB93E10E9481B6EC0114
:102580008EEB93E10E942CB78C01CF3F8FEFD807E1
:1025900039F30F3F8FEF180719F369E773E08DEFF9
:1025A00098E10E9472BC6091BB137091BC134AE029
:1025B00050E08DEF98E10E9452BD6BE37BE08DEF20
:1025C00098E10E9472BC6091B9137091BA134AE00D
:1025D00050E08DEF98E10E9459BDD093BC13C09399
:1025E000BB131093BA130093B91381E08093BD130A
:1025F0000E9429B860934C1570934D1580934E1529
:1026000090934F150AC064E873E08DEF98E1DF9175
:10261000CF911F910F910C949DBCDF91CF911F9191
:102620000F9108954F925F926F927F92AF92BF92F7
:10263000CF92EF92FF920F931F93CF93DF93EC0112
:102640005B0129013A0120910D0240910E02609137
:102650000F0289EF93E10E9459AB85010C5E1F4F79
:10266000809112029E01280F311DA501BE0189EF44
:1026700093E10E9493AC20910A0240910B02609179
:102680000C0289EF93E10E9459AB20910D02409119
:102690000E0260910F0289EF93E10E946DAB80E220
:1026A000C82EE12CF12C85019E01B301A20189EF16
:1026B00093E10E9404B2DF91CF911F910F91FF909F
:1026C000EF90CF90BF90AF907F906F905F904F90C2
:1026D00008954F925F926F927F928F92AF92BF92C6
:1026E000CF92EF92FF920F931F93CF93DF93EC0162
:1026F0007B0129013A0120910D0240910E02609167
:102700000F0289EF93E10E9459AB87010C5E1F4FC6
:10271000809112029E01280F311DA701BE0189EF91
:1027200093E10E9493AC20910A0240910B026091C8
:102730000C0289EF93E10E9459AB20910D02409168
:102740000E0260910F0289EF93E10E946DAB90E25F
:10275000892EA12CB12C2EE2C22E8E0122E0B301D3
:10276000A20189EF93E10E94FDB2DF91CF911F9109
:102770000F91FF90EF90CF90BF90AF908F907F9090
:102780006F905F904F900895AF92BF92CF92DF927B
:10279000EF92FF920F931F93CF93DF93CDB7DEB7E6
:1027A0002C970FB6F894DEBF0FBECDBF61E089EF66
:1027B00093E10E94499089EF93E10E94B9AA89EFC1
:1027C00093E10E949EB32091130234E0239F80196D
:1027D0009109112463E070E00E94FCC4609312022E
:1027E00089EF93E10E94A9B3609112024091130214
:1027F000942F960F990F891B8093110250E05093EC
:1028000098124093971250939A124093991270E045
:102810009A01260F371F30939C1220939B123093FE
:102820009E1220939D128901040F151F1093A01270
:1028300000939F125093A2124093A112D801A60FA9
:10284000B71FB093A412A093A3123093A6122093A3
:10285000A5125D01A40EB51EB092A812A092A712F7
:102860005093AA124093A9126501C60ED71ED092AA
:10287000AC12C092AB12EDEAEE2EE2E1FE2EF701B1
:10288000318320835093B0124093AF1290E0A9019E
:10289000480F591F5093B2124093B1123093B412A3
:1028A0002093B312260F371F280F391F3093B6120B
:1028B0002093B5121093B8120093B7125093BA1226
:1028C0004093B912B093BC12A093BB123093BE12C6
:1028D0002093BD12B092C012A092BF125093C212A8
:1028E0004093C112D092C412C092C3123093C61248
:1028F0002093C51220910D0240910E0260910F02AB
:1029000089EF93E10E946DAB209194124091951252
:102910006091961289EF93E10E9459ABF7014081D3
:1029200051818A01085C1F4F20E431E060E070E0D3
:1029300089EF93E10E9493AC2091941240919512FB
:102940006091961289EF93E10E946DAB20910A028B
:1029500040910B0260910C0289EF93E10E9459AB08
:1029600061E08EEB93E10E9402B462E08EEB93E1B2
:102970000E94CCB764ED77E089EF93E10E9483B3C6
:10298000F70120813181265F3F4F00E010E041E1F7
:1029900050E065E973E089EF93E10E9415B168EBBF
:1029A00073E189EF93E10E9483B3F70120813181C4
:1029B000205E3F4F44E150E061EA73E089EF93E12C
:1029C0000E9415B120910D0240910E0260910F02FC
:1029D00089EF93E10E946DABF701E080F180EE0C8E
:1029E000FF1C80911302E80EF11C66EB73E0CE0130
:1029F00007960E94AEBF60E076E1CE0107960E9486
:102A000074C0BC01CE0101960E940DC0970144E143
:102A100050E0BE016F5F7F4F89EF93E10E94BEB12E
:102A2000CE0101960E9446BFCE0107960E9446BF86
:102A30002C960FB6F894DEBF0FBECDBFDF91CF91BD
:102A40001F910F91FF90EF90DF90CF90BF90AF90CC
:102A50000895EF92FF920F931F93CF93DF93CDB71B
:102A6000DEB72C970FB6F894DEBF0FBECDBF9091A6
:102A70008D132091AD123091AE1280911302220F6E
:102A8000331F281B310900E010E044E150E0992396
:102A900009F4B0C061E174E089EF93E10E9415B1DF
:102AA00064EF71E080E090E00E9458B880918C1350
:102AB000882309F496C020910D0240910E02609186
:102AC0000F0289EF93E10E9459AB4091AD125091F2
:102AD000AE12440F551F80911302481B51098A0101
:102AE0000F5E1F4F20E431E060E070E089EF93E17A
:102AF0000E9493AC64EF71E080E090E00E9458B8CF
:102B000020910A0240910B0260910C0289EF93E13F
:102B10000E9459AB69E278E0CE0107960E94AEBFF1
:102B20002091AD123091AE12220F331F809113020B
:102B3000281B310900E010E044E150E068EB73E04D
:102B400089EF93E10E9415B1809114028823E9F086
:102B500080914F13882319F067EC73E002C06EED8B
:102B600073E0CE0101960E94AEBF60E573E1CE0135
:102B700001960E9474C0BC01CE0107960E94F8BF66
:102B8000CE0101960E9446BF06C06FEE73E0CE01F3
:102B900007960E9420C0E090AD12F090AE12EE0CAD
:102BA000FF1C80911302E81AF108BE01695F7F4F94
:102BB000CE0101960E940DC000E010E0970144E1B3
:102BC00050E0BE016F5F7F4F89EF93E10E94BEB17D
:102BD000CE0101960E9446BFCE0107960E9446BFD5
:102BE0000FC000E010E021E130E04AE050E06CEF7F
:102BF00073E002C06EE074E089EF93E10E9415B1CA
:102C00002C960FB6F894DEBF0FBECDBFDF91CF91EB
:102C10001F910F91FF90EF9008950F931F93182F1E
:102C200020919412409195126091961289EF93E150
:102C30000E9459ABE12FF0E0DF01AA0FBB1FAA0FE2
:102C4000BB1FA556BD4E12960D911C9113972D9149
:102C50003C91EE0FFF1FEE0FFF1FE956FD4E428124
:102C600053816081718189EF93E10E9493AC20913F
:102C70009412409195126091961289EF93E10E940F
:102C80006DAB20910A0240910B0260910C0289EF1A
:102C900093E11F910F910C9459ABCF92DF92EF9279
:102CA000FF920F931F93CF93DF931F921F92CDB785
:102CB000DEB7182F062F61E274E08DEF98E12A83CA
:102CC00049830E949DBC8FEF810F2A814981863004
:102CD00008F055C0602F89EF93E10E9459AB110FA6
:102CE0001250412F50E07A01EE0CFF1CEE0CFF1C3D
:102CF000C70185569D4E7C01FC0102811381015064
:102D00001109208131816A01CC0CDD1CCC0CDD1C49
:102D1000C60189569D4E6C01FC0142815381608140
:102D2000718189EF93E10E944FACF7010281138119
:102D3000025011092081318121503109F60142816F
:102D400053814F5F5F4F608171816F5F7F4F89EF6C
:102D500093E10E944FAC20919412409195126091A2
:102D6000961289EF93E10E946DAB20910D02409184
:102D70000E0260910F0289EF93E10E9459AB6CE261
:102D800074E08DEF98E10F900F90DF91CF911F913C
:102D90000F91FF90EF90DF90CF900C949DBC0F931C
:102DA0001F9390E0FC013197ED32F10508F05FC709
:102DB000EE58FF4F0C944DC580E02FDF809112023A
:102DC000869590E02091991230919A12280F391F20
:102DD0002C5031094091971250919812480F591F69
:102DE0004A50510900E010E062E974E089EF93E194
:102DF0000E9415B180911202869590E0209199125F
:102E000030919A12280F391F4091971250919812C1
:102E1000480F591F4E50510966E374E024C780E003
:102E2000FCDE80911202869590E0209199123091FB
:102E30009A12280F391F2C50310940919712509146
:102E40009812480F591F4651510900E010E06BE3FA
:102E500074E089EF93E10E9415B18091120286958A
:102E600090E02091991230919A12280F391F4091C9
:102E7000971250919812480F591F4650510962E419
:102E800074E0F1C680E0C9DE80911202869590E080
:102E90002091991230919A12280F391F2C50310924
:102EA0004091971250919812480F591F465151095D
:102EB00000E010E06BE374E089EF93E10E9415B14C
:102EC00080911202869590E02091991230919A1289
:102ED000280F391F4091971250919812480F591F8F
:102EE0004A50510965E474E0BEC680E096DE8091E8
:102EF0001202869590E02091991230919A12280F33
:102F0000391F2C5031094091971250919812480F57
:102F1000591F4651510900E010E069E474E089EF5F
:102F200093E10E9415B180911202869590E0209164
:102F3000991230919A12280F391F4091971250918F
:102F40009812480F591F4051510960E574E08BC633
:102F500080E063DE80911202869590E020919912C4
:102F600030919A12280F391F2C5031094091971235
:102F700050919812480F591F4651510900E010E036
:102F800066E574E089EF93E10E9415B18091120229
:102F9000869590E02091991230919A12280F391F4E
:102FA0004091971250919812480F591F485151095A
:102FB0006DE574E058C682E030DE8091120286959D
:102FC00090E02091A1123091A212280F391F2251B6
:102FD000310940919F125091A012480F591F4E5035
:102FE000510900E010E065E674E089EF93E10E948A
:102FF00015B180911202869590E02091A112309136
:10300000A212280F391F2650310940919F1250916A
:10301000A012480F591F4E5051096AE674E089EF1B
:1030200093E10E9415B180911202869590E0209163
:10303000A1123091A212280F391F2A5F3F4F4091F1
:103040009F125091A012480F591F465051096FE628
:1030500074E009C684E0E1DD80911202869590E07B
:103060002091A9123091AA12280F391F2650310938
:103070004091A7125091A812480F591F4E50510964
:1030800000E010E062E774E0EEC584E0C6DD809108
:103090001202869590E02091A9123091AA12280F71
:1030A000391F2C5031094091A7125091A812480F96
:1030B000591F4251510900E010E067E774E089EFC1
:1030C00093E10E9415B180911202869590E02091C3
:1030D000A9123091AA12280F391F4091A7125091BE
:1030E000A812480F591F425151096DE774E0BBC542
:1030F00086E093DD80911202869590E02091B112D6
:103100003091B212280F391F265031094091AF1269
:103110005091B012480F591F4251510900E010E080
:1031200063E874E0A0C586E078DD809112028695A0
:1031300090E02091B1123091B212280F391F265021
:1031400031094091AF125091B012480F591F4651AA
:10315000510900E010E069E874E085C584E05DDDB8
:1031600080911202869590E02091A9123091AA12C6
:10317000280F391F265031094091A7125091A812EB
:10318000480F591F4251510900E010E060E974E016
:103190006AC588E042DD80911202869590E0209118
:1031A000B9123091BA12280F391F2C5031094091B1
:1031B000B7125091B812480F591F4A50510900E0F8
:1031C00010E066E974E089EF93E10E9415B1809107
:1031D0001202869590E02091B9123091BA12280F10
:1031E000391F4091B7125091B812480F591F4650DD
:1031F000510968EF74E037C588E00FDD8091120255
:10320000869590E02091B9123091BA12280F391F9B
:103210002C5031094091B7125091B812480F591FE4
:103220004A50510900E010E066E974E089EF93E14B
:103230000E9415B180911202869590E02091B912FA
:103240003091BA12280F391F4091B7125091B8121D
:10325000480F591F4E5051096FEE74E004C582E0CB
:10326000DCDC80911202869590E02091A1123091D1
:10327000A212280F391F2C50310940919F125091F2
:10328000A012480F591F4C50510900E010E06AE9A4
:1032900074E089EF93E10E9415B180911202869546
:1032A00090E02091A1123091A212280F391F409175
:1032B0009F125091A0122CC088E0AFDC80911202C6
:1032C000869590E02091B9123091BA12280F391FDB
:1032D0002C5031094091B7125091B812480F591F24
:1032E0004C50510900E010E064EA74E089EF93E18A
:1032F0000E9415B180911202869590E02091B9123A
:103300003091BA12280F391F4091B7125091B8125C
:10331000480F591F4C50510982C086E07EDC8091D5
:103320001202869590E02091B1123091B212280FCE
:10333000391F265031094091AF125091B012480FF9
:10334000591F4E50510900E010E069EA74E08BC447
:103350008AE063DC80911202869590E02091C11290
:103360003091C212280F391F225131094091BF12EA
:103370005091C012480F591F4E50510900E010E003
:1033800065E674E01AC08AE048DC809112028695F6
:1033900090E02091C1123091C212280F391F2251A2
:1033A00031094091BF125091C012480F591F4E5021
:1033B000510900E010E063EB74E089EF93E10E94B3
:1033C00015B180911202869590E02091C112309142
:1033D000C212280F391F265031094091BF12509157
:1033E000C012480F591F4E5051096EEA74E089EF20
:1033F00093E10E9415B180911202869590E0209190
:10340000C1123091C212280F391F2A5F3F4F4091DD
:10341000BF125091C012480F591F4E5051096FE909
:1034200074E021C48AE0F9DB80911202869590E075
:103430002091C1123091C212280F391F2C5031092E
:103440004091BF125091C012480F591F4E50510960
:1034500000E010E062E774E089EF93E10E9415B1AB
:1034600080911202869590E02091C1123091C21293
:10347000280F391F4091BF125091C012480F591F99
:103480004A50510963E373E0EEC382E0C6DB8091EA
:103490001202869590E02091A1123091A212280F7D
:1034A000391F2C50310940919F125091A012480FA2
:1034B000591F4A50510900E010E068EB74E089EFB1
:1034C00093E10E9415B180911202869590E02091BF
:1034D000A1123091A212280F391F40919F125091D2
:1034E000A012D5C188E099DB80911202869590E008
:1034F0002091B9123091BA12280F391F2C5031097E
:103500004091B7125091B812480F591F4A505109B3
:1035100000E010E062EC74E0A8C184E07EDB809102
:103520001202869590E02091A9123091AA12280FDC
:10353000391F2C5031094091A7125091A812480F01
:10354000591F4A50510900E010E068EB74E089EF20
:1035500093E10E9415B180911202869590E020912E
:10356000A9123091AA12280F391F4091A712509129
:10357000A8122CC08AE051DB80911202869590E05F
:103580002091C1123091C212280F391F2C503109DD
:103590004091BF125091C012480F591F4A50510913
:1035A00000E010E062EC74E089EF93E10E9415B155
:1035B00080911202869590E02091C1123091C21242
:1035C000280F391F4091BF125091C012480F591F48
:1035D0004251510966EC74E046C382E01EDB8091E3
:1035E0001202869590E02091A1123091A212280F2C
:1035F000391F2C50310940919F125091A012480F51
:10360000591F4A50510900E010E068EB74E089EF5F
:1036100093E10E9415B180911202869590E020916D
:10362000A1123091A212280F391F40919F12509180
:10363000A0122CC088E0F1DA80911202869590E009
:103640002091B9123091BA12280F391F2C5031092C
:103650004091B7125091B812480F591F4A50510962
:1036600000E010E062EC74E089EF93E10E9415B194
:1036700080911202869590E02091B9123091BA1291
:10368000280F391F4091B7125091B812480F591F97
:10369000405151096CEC74E0E6C284E0BEDA8091DE
:1036A0001202869590E02091A9123091AA12280F5B
:1036B000391F225131094091A7125091A812480F89
:1036C000591F4A50510900E010E068EB74E07EC0D9
:1036D0008AE0A3DA80911202869590E02091C112CF
:1036E0003091C212280F391F225131094091BF1267
:1036F0005091C012480F591F4A50510900E010E084
:1037000062EC74E089EF93E10E9415B1809112029E
:10371000869590E02091C1123091C212280F391F76
:10372000265031094091BF125091C012480F591FC5
:103730004A50510966E974E089EF93E10E9415B19E
:1037400080911202869590E02091C1123091C212B0
:10375000280F391F2A5F3F4F4091BF125091C0126E
:1037600063C086E05ADA80911202869590E020913B
:10377000B1123091B212280F391F265031094091F1
:10378000AF125091B012480F591F4251510900E039
:1037900010E066ED74E067C284E03FDA80911202C7
:1037A000869590E02091A9123091AA12280F391F16
:1037B000225131094091A7125091A812480F591F68
:1037C0004A50510900E010E06BED74E089EF93E19D
:1037D0000E9415B180911202869590E02091A91265
:1037E0003091AA12280F391F265031094091A71293
:1037F0005091A812480F591F4A50510966E974E0C8
:1038000089EF93E10E9415B180911202869590E0B4
:103810002091A9123091AA12280F391F2A5F3F4F19
:103820004091A7125091A812480F591F4E505109AC
:1038300061ED74E018C288E0F0D98091120286959B
:1038400090E02091B9123091BA12280F391F2C50F4
:1038500031094091B7125091B812480F591F4A5080
:10386000510900E010E06BED74E089EF93E10E94F4
:1038700015B180911202869590E02091B912309195
:10388000BA12280F391F4091B7125091B812480F41
:10389000591F425151096CEB74E0E5C182E0BDD97A
:1038A00080911202869590E02091A1123091A2128F
:1038B000280F391F2C50310940919F125091A012AE
:1038C000480F591F4A50510900E010E06BED74E0B9
:1038D00089EF93E10E9415B180911202869590E0E4
:1038E0002091A1123091A212280F391F40919F12EE
:1038F0005091A012480F591F4A5051096FED74E0C2
:10390000B2C182E08AD980911202869590E020911E
:10391000A1123091A212280F391F2C503109409169
:103920009F125091A012480F591F4A50510900E0B0
:1039300010E068EB74E089EF93E10E9415B180918B
:103940001202869590E02091A1123091A212280FC8
:10395000391F40919F125091A0122CC088E05DD970
:1039600080911202869590E02091B9123091BA129E
:10397000280F391F2C5031094091B7125091B812BD
:10398000480F591F4A50510900E010E062EC74E002
:1039900089EF93E10E9415B180911202869590E023
:1039A0002091B9123091BA12280F391F4091B712E5
:1039B0005091B812480F591F4A50510963EE74E0F4
:1039C00052C184E02AD980911202869590E020911C
:1039D000A9123091AA12280F391F2C503109409199
:1039E000A7125091A812480F591F4A50510900E0E0
:1039F00010E068EB74E089EF93E10E9415B18091CB
:103A00001202869590E02091A9123091AA12280FF7
:103A1000391F4091A7125091A8122CC08AE0FDD8FE
:103A200080911202869590E02091C1123091C212CD
:103A3000280F391F2C5031094091BF125091C012EC
:103A4000480F591F4A50510900E010E062EC74E041
:103A500089EF93E10E9415B180911202869590E062
:103A60002091C1123091C212280F391F4091BF120C
:103A70005091C012480F591F4A50510967EE74E027
:103A8000F2C082E0CAD880911202869590E020911F
:103A9000A1123091A212280F391F2C5031094091E8
:103AA0009F125091A012480F591F4A50510900E02F
:103AB00010E068EB74E089EF93E10E9415B180910A
:103AC0001202869590E02091A1123091A212280F47
:103AD000391F40919F125091A0122CC088E09DD8B0
:103AE00080911202869590E02091B9123091BA121D
:103AF000280F391F2C5031094091B7125091B8123C
:103B0000480F591F4A50510900E010E062EC74E080
:103B100089EF93E10E9415B180911202869590E0A1
:103B20002091B9123091BA12280F391F4091B71263
:103B30005091B812480F591F4A5151096BEE74E069
:103B400092C084E06AD880911202869590E020911C
:103B5000A9123091AA12280F391F2C503109409117
:103B6000A7125091A812480F591F4A50510900E05E
:103B700010E068EB74E089EF93E10E9415B1809149
:103B80001202869590E02091A9123091AA12280F76
:103B9000391F4091A7125091A8122CC08AE03DD83D
:103BA00080911202869590E02091C1123091C2124C
:103BB000280F391F2C5031094091BF125091C0126B
:103BC000480F591F4A50510900E010E062EC74E0C0
:103BD00089EF93E10E9415B180911202869590E0E1
:103BE0002091C1123091C212280F391F4091BF128B
:103BF0005091C012480F591F4651510964EF74E0AB
:103C000032C080E00AD880911202869590E020911F
:103C1000991230919A12280F391F2C503109409176
:103C2000971250919812480F591F4851510900E0BE
:103C300010E06BEF74E089EF93E10E9415B1809181
:103C40001202869590E02091991230919A12280FD5
:103C5000391F4091971250919812480F591F4651A1
:103C6000510963E075E089EF93E10E9415B11F915E
:103C70000F910895CF93DF93EB012A813B81FC01E3
:103C8000338322834C815D816E817F8144835583A0
:103C900066837783488559856A857B854087518708
:103CA000628773872DE0FE013C96DC011C96019033
:103CB0000D922A95E1F7298D3A8DFC01328F218FE3
:103CC000DF91CF910895EF92FF920F931F93CF93BF
:103CD000DF93CDB7DEB7E7970FB6F894DEBF0FBE20
:103CE000CDBF7C018B0141E06EE873E1CE014C96C3
:103CF0000E945B6ECE014C960E949F6B882399F1C7
:103D0000CE014C960E94246BBC01C8010E94EAC0FF
:103D1000882359F160E675E08DEF98E10E949DBC23
:103D2000CE014C960E948D6B41E06EE873E1CE01AE
:103D300001960E945B6EBE016F5F7F4FCE014C9675
:103D400099DFCE014C960E949F6B882341F0CE01F3
:103D50004C960E94246BBC01C8010E9420C0CE0179
:103D60004C960E948D6B21E001C020E0CE014C9664
:103D70002FAB0E948D6B2FA9222309F4B4CFB80179
:103D8000C7010E9421BFC701E7960FB6F894DEBFB6
:103D90000FBECDBFDF91CF911F910F91FF90EF909C
:103DA0000895EF92FF920F931F93CF93DF93CDB7B8
:103DB000DEB7EC970FB6F894DEBF0FBECDBF7C0127
:103DC0008B0169E278E0CE01C7960E94AEBF41E068
:103DD0006EE873E1CE014C960E945B6ECE014C966C
:103DE0000E949F6B882389F0CE014C960E94246B21
:103DF000BC01C8010E94EAC0882339F06CE675E076
:103E00008DEF98E10E949DBC48C0CE014C960E9467
:103E1000246BBC01CE01C7960E9420C061E775E00B
:103E20008DEF98E10E9472BCBE01695C7F4F8DEFFF
:103E300098E10E948DBCCE014C960E948D6B41E0B2
:103E40006EE873E1CE0101960E945B6EBE016F5F6A
:103E50007F4FCE014C960EDFCE014C960E949F6B99
:103E60008823D9F0CE014C960E94246BBC01C80176
:103E70000E94EAC0882339F0BE01695C7F4FC80107
